:0300000002352B9B
:0C352B0078FFE4F6D8FD7581550235727A
:1013A10020000A3C2E2E2E3E004950436F6E6E6582
:1013B10063745245510A004950436F6E6E65637400
:1013C100000A49504E6F41434B210A003E432C56BF
:1013D1002C43432CC0E4E0EFF2E5F020D1E8EDEA44
:1013E100EEEC49500A003E432C4D41432C2530324E
:1013F10062583A25303262583A25303262583A25DD
:10140100303262583A25303262583A2530326258C9
:101411002C4D414320E0E4F0E5F10A003E432C5617
:1014210045522C20332E3220EEF2202573202573D5
:101431002CC2E5F0F1E8FF20495020ECEEE4F3EB9B
:10144100FF0A0044656320313920323030380031E1
:10145100363A31313A3437003E432C4C442C505209
:101461004F473A202020202020202020202020200B
:10147100202020202020202020202020202020206B
:10148100202020202020202020202020202020205B
:10149100202020202020202020202020202020204B
:1014A10020202020202020202CC4E0F2E020EFF09A
:1014B100EEF8E8E2EAE828F4E0E9EB290A003E2A3E
:1014C1002C312CCEF1EDEEE2EDFBE520EFE0F0E08A
:1014D100ECE5F2F0FB20F1E5F2E5E2EEE3EE20E8E7
:1014E100EDF2E5F0F4E5E9F1E00A003E412C41308E
:1014F100312C2562752E2562752E2562752E256289
:10150100752C495020E0E4F0E5F120E0E4E0EFF251
:10151100E5F0E00A003E412C4130322C2562752E67
:101521002562752E2562752E2562752C495020E0A5
:10153100E4F0E5F120EEF1ED2E20F1E5F0E2E5F049
:10154100E00A003E412C4130332C2562752E256284
:10155100752E2562752E2562752C495020E0E4F028
:10156100E5F120F0E5E72E20F1E5F0E2E5F0E00A13
:10157100003E412C4130342C2562752E2562752E9A
:101581002562752E2562752CCCE0F1EAE020F1E5AB
:10159100F2E80A003E412C4130352C2562752E259A
:1015A10062752E2562752E2562752CD8EBFEE70A31
:1015B100003E2A2C312CC4EEEF2E20EFE0F0E0ECBF
:1015C100E5F2F0FB20F1E5F2E5E2EEE3EE20E8EDF5
:1015D100F2E5F0F4E5E9F1E00A003E422C53303146
:1015E1002C2562752CC6E4E0F2FC20E7E0EFF0EE7A
:1015F100F1E020F1EEE5E4E8EDE5EDE8FF20EEF2C3
:1016010020F1E5F0E2E5F0E00A003E422C533032F1
:101611002C2562752CCEE1ECE5ED20F120F1E5F011
:10162100E2E5F0EEEC20E1E5E720EAE2E8F2E0EDC8
:10163100F6E8E90A003E422C5330332C2562752C22
:10164100CFE5F0E5E7E0EFF3F1EA20EFF0E820EF96
:10165100EEF2E5F0E520F1E2FFE7E820F120F1E527
:10166100F0E2E5F0EEEC0A003E454E440A000A4481
:10167100756D7058202020202030302030312030EE
:10168100322030332030342030352030362030378E
:101691002030382030392030412030422030432062
:1016A1003044203045203046000A3A003A20000AF2
:1016B100000A44756D7044202020202030302030F5
:1016C1003120303220303320303420303520303654
:1016D100203037203038203039203041203042202E
:1016E100304320304420304520304600457272207E
:1016F1006B657900526420656570726F6D0A0052E6
:1017010064204D454D0A00526420436F64650A0010
:10171100577269746520436F64650A004465627598
:10172100674950204F4E0A00446562756749502051
:101731004F46460A00446562756755736572204FCE
:101741006E0A00446562756755736572204F46469F
:101751000A0044656275674D7367204F6E0A004445
:10176100656275674D7367204F46460A00436F6E89
:10177100666967206C6F636B210A0057722065658B
:1017810070726F6D0A002053617665206565707215
:101791006F6D210A00457272204D414321004C6F4B
:1017A10061643E3E002A003C4130313D003C413005
:1017B100323D003C4130333D003C4130343D003C42
:1017C1004130353D003C21003C5330313D003C531C
:1017D10030323D003C5330333D003C5330353D0009
:0617E1003C5330363D00D0
:063D5000015200015000C9
:103DAE00C28E438910E4F58B758DB8D2ABD28E22BC
:03001B0002349B11
:10349B00C0E0C083C082C0D0C28E758B00758DB862
:1034AB00201E0675A61E75A6E10550D21AE55260C0
:1034BB00020552E551D39401400215510555E555CE
:1034CB00540F7048D226E555543F7012D2189066AF
:1034DB008BE0600A04F0E0D394B44002D21E9066F5
:1034EB0086E0600204F0906104E0600214F09066E4
:1034FB008CE0D394014003E014F0301D020553E53A
:10350B0054D394644004D21E80020554E54FD394E7
:10351B00014002154FD28ED0D0D082D083D0E03272
:10086900C291C290D2B5C2237D027C007F07123D9E
:10087900338F27E527646060097D017F60123CCED4
:10088900D223E4FDFC7F0B123D338F27E52730E6A9
:10089900097D04E4FF123CF2D2237D017C007F072D
:1008A900123D338F27E5277008FD7FFF123CCED21A
:1008B90023302303126000C288C2A8C2AA75890026
:1008C90012385390633EE0B4FA06A3E064CE607B2D
:1008D900E4F52774362527F582E43463F583E4F0DB
:1008E9000527E527B443EC90633E74FAF0A374CE70
:1008F900F0A374CCF0906344740AF0E4A3F0A30469
:10090900F0A3F090633A74FFF0A3F0A3F0E4A3F02E
:10091900906355740AF0E4F527E5272401FFE433D1
:10092900FE74362527F582E43463F583E0FD123C35
:10093900AA0527E527C3944340DFE4F5A775A61E5A
:1009490075A6E1907FF0F0A3F080FE9063497403EF
:10095900F0A374CCF0E4906348F01231B7C2B51239
:1009690033EDC21E123B2FD223C225C224906576D5
:100979007408F09062B47424F0E4A3F090633EE04C
:100989009062B6F090633FE09062B7F0906340E008
:100999009062B8F0906341E09062B9F0906342E0F0
:1009A9009062BAF0906343E09062BBF0755101E444
:1009B900906577F0C21FC220C221C222202318AF3E
:1009C90027FE7D03122E53E4FF12333D7E137FA1D0
:1009D900E4FBFDFC12287390668BE060037401F060
:1009E900E4906104F0F553906575F0F554123DAE4D
:1009F90075A70775A61E75A6E1D2AFE4F5549061F7
:100A090004E07003122A7E90668CE06401701D90E8
:100A190080007410F09080A874FFF0A3F0A3F0A3F5
:100A2900F0E490668CF0D223C224C225908008E0BD
:100A3900F52730E405D21F7410F0E52730E508D218
:100A4900219080087420F0E52730E608D2209080B4
:100A5900087440F0E553C394034019908002E4F010
:100A6900908001F0908000F0E55394064006E4F58B
:100A790053123B2F9080A0E0700312394B9080B83D
:100A8900E070031238D19080D0E07003123A799067
:100A99008000E07013301F1012297A906331EFF053
:100AA900D394004003120026908002E070069080E3
:100AB90000E06005D21D020A04C21DE4F5539061ED
:100AC90004E06003020A04202312906578E0600CB8
:100AD9007E137FA3122D6BE4906578F030211212FA
:100AE9002464906331EFF0D394004005E0FF123D98
:100AF900DD202003020C7A1222DD906331EFF070C1
:100B090003020A04906375E054BF247F7003020B4B
:100B1900E3147003020BBB24026003020C1C2023A4
:100B2900077E137FAA122D6B202703020C7A90638C
:100B39004DE07006906351E06067906682E0FF9037
:100B4900634DE0B50724906683E0FE90634EE0B5FF
:100B59000618906684E0FE90634FE0B5060C906637
:100B690085E0FE906350E06E6037906351E06F60FE
:100B790003020C7A906683E0FF906352E06F600392
:100B8900020C7A906684E0FF906353E06F60030281
:100B99000C7A906685E0FF906354E06F6003020C65
:100BA9007AC21B9065777401F012001E755101021B
:100BB9000C7A90668BE060037401F090667AE0FF2E
:100BC900906377E06F6003020C7A90667AE004F034
:100BD900E4F551906575F0020C7A301B03020C7A2A
:100BE900906344E07003020A04906355740AF0129A
:100BF9003DD3D21BE4F551906575F090668604F0FB
:100C0900E4906679F0A3F02023677E137FB8122D54
:100C19006B805E90668BE060037401F0301B52902C
:100C29006375E020E74B906377E0FF906679E0FE1B
:100C39006F600D906681E07007EE146F703380135A
:100C4900906679E004F0906331E0FFD394044003A7
:100C5900123AD59060007482F0A37401F090637722
:100C6900E0906002F07E607F007D0312363E020A4A
:100C790004201B03020D92E5517068122141EF60B7
:100C8900237E647F75906476E02404FD12363E90DD
:100C99006681E07009906355E0F551020A04E4F5B4
:100CA90051020A04906686E0D3943C4036906681EE
:100CB900E0703090668604F0123281E4906475F039
:100CC900A37412F090667AE0906477F0A374FDF053
:100CD90090610563A20190647963A2017F12121EDB
:100CE9008F809E123D9A8F27E527B40115906000E9
:100CF9007483F0E4A3F07E607F007D0212363E0229
:100D09000A04E527D39401401C9060007483F0A382
:100D19007401F0E52724FEA3F07E607F007D0312B5
:100D2900363E020A04E55164016003020A04906533
:100D390075E004F02023077E137FC2122D6B9063A8
:100D490055E0C394C85004E02432F0906575E0C3BF
:100D59009405400DC21BE4906577F012001E020A4B
:100D6900047C667D82906349E0FAA3E0FB7F02126E
:100D790037CF7E647F75906476E02404FD12363E99
:100D8900906355E0F551020A04E5516401600302DC
:100D99000A04906577E014604624FE6042147003EB
:100DA900020E8524046003020A04E4F55320271384
:100DB9009065777404F0906575E05401F075510100
:100DC900020A049080027410F0E4906577F090654F
:100DD9007504F07551FA90668274FFF0020A049066
:100DE9006682E07003020E6F9064757480F09064FF
:100DF900777401F0E4A3F0A304F0A37430F0A374B2
:100E09007BF0E4F527747C2527F582E43464F583C7
:100E1900747DF0747D2527F582E43464F583E4F06C
:100E2900E5272407906476F07C667D82906349E02B
:100E3900FAA3E0FB7F021237CF7E647F75E5272492
:100E490009FD12363E906681E0601B123DD3D21B2C
:100E5900E4F551906575F090668604F0E490667942
:100E6900F0A3F0020A04302707E4906577F08006C2
:100E79009065777404F07551FA020A04908002743F
:100E890010F0755105906575E06401FFF090657784
:100E99007401F0EF7019906351E06013FCA3E0FD59
:100EA900A3E0FEA3E0FF906682121C5B020A049095
:100EB900634DE0FCA3E0FDA3E0FEA3E0FF906682A2
:080EC900121C5B020A0480FE0A
:010ED10022FE
:10002600906376E0B444047F0180027F009063759C
:10003600E0B447047E0180027E00EE5F604A906372
:100046003EE0906377F090633FE0906378F09063D2
:1000560040E0906379F0906341E090637AF09063BA
:1000660042E090637BF0906343E090637CF09063A2
:10007600767452F09062AE63A2019080A863A201EA
:100086007F06121E8F02085F906331E0C39408500A
:100096000302086890633EE0FF906377E06F6003B9
:1000A60002086890633FE0FF906378E06F600302A8
:1000B6000868906340E0FF906379E06F6003020890
:1000C60068906341E0FF90637AE06F60030208681E
:1000D600906342E0FF90637BE06F600302086890E4
:1000E6006343E0FF90637CE06F60030208689063FF
:1000F60076E06444701A9080A8E0B4FF139062AE74
:1001060063A2019080A863A2017F06121E8F801051
:100116009062B2E09080ACF09062B3E09080ADF077
:1001260090668BE060037401F090668C7464F090C6
:1001360063767452F0906375E0646D600302026941
:100146007BFF7A1379CD1218497BFF7A1379E790F2
:10015600633EE0F530A3E0F531A3E0F532A3E0F528
:1001660033A3E0F534A3E0F5351218497530FF7571
:1001760031147532447533FF7534147535507BFF71
:100186007A14791D1218497BFF7A14795912184985
:100196007BFF7A1479BF1218497BFF7A1479EC90A9
:1001A6006344E0F530A3E0F531A3E0F532A3E0F5D2
:1001B600331218497BFF7A15791690634DE0F530B6
:1001C600A3E0F531A3E0F532A3E0F5331218497B3D
:1001D600FF7A157944906351E0F530A3E0F531A339
:1001E600E0F532A3E0F5331218497BFF7A157972F0
:1001F60090633AE0F530A3E0F531A3E0F532A3E0F1
:10020600F5331218497BFF7A157995906336E0F538
:1002160030A3E0F531A3E0F532A3E0F53312184937
:100226007BFF7A1579B21218497BFF7A1579DBA222
:1002360027E433F5301218497BFF7A16790B90665E
:1002460081E0F5301218497BFF7A16793690668B75
:10025600E0F5301218491230EB7BFF7A16796912F5
:10026600184922906375E0644C70737E167F6FFBAD
:10027600FDFC12287390637DE0F528A3E0F529E4E0
:10028600F52BE52890637FF0A3E529F07E167FAA7B
:100296007C637D7F7B02122873E4F52A852982859B
:1002A6002883E0FF747F252AF582E43463F583EF23
:1002B600F00529E52970020528052AE52AB410DC8F
:1002C6007E167FAD7C637D7F7B10122873052BE540
:1002D6002BC3941040AC7E167FB0122D6B22906318
:1002E60075E0646C7060F52C7E167FB2FBFDFC1227
:1002F6002873E4F52BE490637FF0A3E52CF07E16DB
:100306007FAA7C637D7F7B02122873E4F52AA82CE2
:10031600E6FF747F252AF582E43463F583EFF00562
:100326002C052AE52AB410E67E167FAD7C637D7F18
:100336007B10122873052BE52BC3940840B77E1655
:100346007FB0122D6B22906375E0644B7061F52AC5
:100356007467252AF582E43463F583E060327467B6
:10036600252AF582E43463F583E0F4602374672577
:100376002AF582E43463F583E0FF747D252AF5824D
:10038600E43463F583E0B50710052AE52AB408C00E
:100396009061047432F002085F9063757421F03046
:1003A600230302085F7E167FED122D6B02085F9015
:1003B6006375E0B4521A2023077E167FF5122D6B63
:1003C6009063757472F07E637F757D081235B7226F
:1003D600906375E0644970452023077E177F0012FD
:1003E6002D6B90637DE0F528A3E0F529E4F52A85D9
:1003F6002982852883E0FF747F252AF582E4346309
:10040600F583EFF00529E52970020528052AE52A76
:10041600B480DC7E637F757D8A1235B72290637562
:10042600E0644370462023077E177F08122D6B90E9
:10043600637DE0F528A3E0F529E4F52A8529828580
:100446002883E493FF747F252AF582E43463F583D9
:10045600EFF00529E52970020528052AE52AB4806A
:10046600DB7E637F757D8A1235B722906375E06403
:100476005A70532023077E177F11122D6B90637DD0
:10048600E0F528A3E0F5297C637D7F7B80AF29AE6C
:1004960028123C76E4F52A852982852883E493FF91
:1004A600747F252AF582E43463F583EFF00529E5A8
:1004B6002970020528052AE52AB480DB7E637F754C
:1004C6007D8A1235B722906375E0644460030205A5
:1004D6005D90637DE0FF6444700302085FEFB43112
:1004E6000CC2237E177F1D122D6B02085F90637D61
:1004F600E0B4300CD2237E177F29122D6B02085FE1
:1005060090637DE0B4320CD2247E177F36122D6BB9
:1005160002085F90637DE0B4330CC2247E177F44EB
:10052600122D6B02085F90637DE0B4340CD2257EF9
:10053600177F53122D6B02085F90637DE0B4350C74
:10054600C2257E177F60122D6B02085F90637DE0E7
:10055600FF123DDC02085F906104E0701320230760
:100566007E177F6E122D6B9063757421F002085F03
:100576009061047432F0906375E0FFB45104C2AF29
:1005860080FEEF645770452023077E177F7C122D6F
:100596006B90637EE0906331F0E4F52A906331E07E
:1005A600FFE52AC39F400302085F747F252AF58270
:1005B600E43463F583E0FF90637DE0252A24ADF5FE
:1005C60082E43461F583EFF0052A80D0906375E00C
:1005D600645360030206802023077E177F87122D4F
:1005E6006B90633EE0FF9061B6E06F703C90633FB6
:1005F600E0FF9061B7E06F7030906340E0FF90617C
:10060600B8E0B50724906341E0FF9061B9E0B50713
:1006160018906342E0FF9061BAE0B5070C9063431F
:10062600E0FF9061BBE06F60169063757421F03057
:10063600230302085F7E177F96122D6B02085FE484
:10064600F52AE4F554AF2AFE74AD252AF582E43482
:1006560061F583E0FD123CAA052AE52AC394FE4013
:10066600E1C2AFE4907FF0F0A3F0907FFD74AAF0B2
:10067600A374FFF0A37455F080FE906375E0644F99
:10068600704C90637DE0F528A3E0F529E52945281F
:10069600700A2023077E177F9F122D6B2023077E6B
:1006A600177FA6122D6BE4F52A747F252AF582E4BE
:1006B6003463F583E0852982852883F00529E529B9
:1006C60070020528052AE52AB480DE02085F9063D9
:1006D60075E0FFB4452190637DE0FDA3E0907FF0D7
:1006E600CDF0A3EDF0C2AF907FFD74AAF0A374FF26
:1006F600F0A37455F080FEEF64656003020868900D
:10070600637DE0FFA3E0907FF0CFF0A3EFF0E4F588
:1007160028F529D3907FF1E09529907FF0E0952880
:100726004020E4F5542529FFE5283401FE85298279
:10073600852883E0FD123CAA0529E52970020528D3
:1007460080D17E177FA81236C5EF4E6020120003B7
:10075600906344EFF0120003906345EFF01200033C
:10076600906346EFF0120003906347EFF07E177F29
:10077600AE1236C5EF4E602012000390634DEFF0C7
:1007860012000390634EEFF012000390634FEFF0F8
:10079600120003906350EFF07E177FB41236C5EF58
:1007A6004E6020120003906351EFF0120003906335
:1007B60052EFF0120003906353EFF01200039063C0
:1007C60054EFF07E177FBA1236C5EF4E6020120046
:1007D6000390633AEFF012000390633BEFF01200D0
:1007E6000390633CEFF012000390633DEFF07E1739
:1007F6007FC01236C5EF4E6020120003906336EFBD
:10080600F0120003906337EFF0120003906338EFA5
:10081600F0120003906339EFF0E4F52AE4F554E5AD
:100826002A2401FFE433FE7436252AF582E4346374
:10083600F583E0FD123CAA052AE52AC3944340DC71
:10084600C2AFE4907FF0F0A3F0907FFD74AAF0A30E
:1008560074FFF0A37455F080FE7E637F757D0812E9
:0208660035B7A4
:01086800226D
:103C0900AE07EEC39430400BEED394395005EE2441
:103C1900D0FF22EEC39461400BEED394665005EEBB
:103C290024A9FF22EEC39441400BEED394465005DC
:083C3900EE24C9FF22AF0622B0
:103D6C009062ADE004F070069062ACE004F09062FA
:0A3D7C00ACE0FEA3E0FF123D1622AA
:10000300123D6C123C09EFC454F0FEC006123D6C65
:08001300123C09D0E02FFF228E
:103A1C00E4906AC2F0123D6C906AC3EFF0C394302C
:103A2C004018E0FFD394395011906AC2E02405F598
:103A3C0082E43461F583EFF08011906AC2E02405D2
:103A4C00F582E43461F583E4F0800C906AC2E00402
:103A5C00F0E0D3940840BE752B00752C00752D003A
:0C3A6C00E4F52E7B017A617905121F9DA4
:013A7800222B
:0436C5008E2D8F2E89
:1036C9009062ACE4F0A374FFF0123D6CEF606EF40D
:1036D900606B852E82852D83E493B507EC752F01E8
:1036E900E52E252FF582E4352DF583E493602590A9
:1036F90062ADE0252FFF9062ACE03400FE123D166A
:10370900E52E252FF582E4352DF583E493B50704DD
:10371900052F80CCE52E252FF582E4352DF583E4A0
:103729009370A6E52F24FFFFE434FFFE9062ADE01D
:103739002FF09062ACE03EF07E007F0122E4FEFFB4
:01374900225D
:1031B7007E177FC61236C5EF4E70037F01227E173A
:1031C7007FC91236C5EF4E600C123D6CEF24D02438
:1031D700FF92278002D2277E177FCF1236C5EF4E88
:1031E700600C123D6CEF24D0906681F08005E4906E
:1031F7006681F07E177FD51236C5EF4E600C123D03
:103207006CEF24D090668BF08005E490668BF07E9F
:10321700177FDB1236C5EF4E600C123D6CEF24D0E2
:1032270024FF92198002C21990633E63A20190663F
:103237007B63A2017F06121E8F30193B7E177FE149
:103247001236C5EF4E603012000390667BEFF01226
:10325700000390667CEFF012000390667DEFF0129A
:10326700000390667EEFF012000390667FEFF01286
:0A3277000003906680EFF07F002254
:103B8900906576E0C3947C503D906576E0FE04F044
:103B990074B42EF582E43462F583EFF0BF0A2790FE
:103BA9006576E0FF04F074B42FF582E43462F5839E
:103BB900E4F0906576E0FF12374A9065767408F074
:073BC9009062B5E004F02258
:100ED2003E2A2C312CCFE0F0E0ECE5F2F0FB20E0F2
:100EE200F1E8EDF5F0EEEDEDEEE3EE20EFEEF0F2EF
:100EF200E02E20D0E5E6E8EC20F0E0E1EEF2FB2087
:100F02002D20EFE0EAE5F2EDFBE920EFEE2055447B
:100F12005020E820EAE2E0E7E8EFEEF2EEEAEEE265
:100F2200FBE920EFEE205443500A003E432C4B30A5
:100F3200362C25732CD2E5EAF3F9E8E920F0E5E650
:100F4200E8EC0A003E4C2C4930312C256C752CD132
:100F5200EAEEF0EEF1F2FC20EEE1ECE5EDE02C350C
:100F6200302C3130302C3330302C3630302C313282
:100F720030302C323430302C343830302C3936305A
:100F8200302C31393230302C33383430302C353744
:100F92003630302C3131353230300A003E422C4965
:100FA20030322C2562752CD3EFF0E0E2EBE5EDE870
:100FB200E520EFEEF2EEEAEEEC20EFF0E820EFE5CE
:100FC200F0E5E4E0F7E520285254532D4354532929
:100FD2000A003E532C4930332C2562752CC7E0E4BD
:100FE200E5F0E6EAE020F1F2E0F0F2E020EFE5F0F1
:100FF200E5E4E0F7E8282A3130ECF1290A003E4224
:101002002C4930342C2562752CD0E5E6E8EC20EF33
:10101200E5F0E5E4E0F7E8203720E1E8F20A003EF7
:10102200422C4930352C2562752CCFE5F0E5E4E001
:10103200F7E020F120EAEEEDF2F0EEEBFCEDFBEC56
:1010420020E1E8F2EEEC0A003E422C4930362C2533
:1010520062752CCAEEEDF2F0EEEBFCEDFBE920E15D
:10106200E8F2202D20F7E5F2EDEEF1F2FC0A003E67
:10107200422C415030372C2562752CC6E4E0F2FC3C
:1010820020EAE2E8F2E0EDF6E8FE20EEF220F3F1EB
:10109200F2F0EEE9F1F2E2E00A003E422C41503079
:1010A200382C2562752CCAE2E8F2E8F0EEE2E0F2B2
:1010B200FC20EFE0EAE5F2FB20EEF220F3F1F2F0A1
:1010C200EEE9F1F2E2E00A003C21003C4930313D18
:1010D200003C4930323D003C4930333D003C493010
:1010E200343D003C4930353D003C4930363D003C02
:1010F200415030373D003C415030383D000A536585
:101102006E64205061636B65743A20000A53656E09
:1011120064204B56543A20000AC1F3F4E5F020E76C
:10112200E0EDFFF221000A435243206572726F72B2
:1011320021202020000ACEF2E2E5F7E0FE20EDE0D9
:1011420020E7E0E3F0F3E7EAF321000A52656320C7
:101152004B5654000A526563206F6B2120202020D9
:10116200202000496E69745443500A004C6973741C
:10117200656E5443500A00534F434B5F5443505FD4
:1011820045535441424C49534845440A000A2D3EB6
:1011920020000A3C2D2000544350005544500000CA
:1011A200112332465765748C9DAFBECADBE9F81035
:1011B200013322564775649C8DBFAEDACBF9E82124
:1011C20030021367764455ADBC8E9FEBFAC8D93115
:1011D20020120377665445BDAC9E8FFBEAD8C94204
:1011E20053617004152736CEDFEDFC8899ABBA52F5
:1011F20043716014053726DECFFDEC9889BBAA63E4
:1012020072405125340617EFFECCDDA9B88A9B73D4
:1012120062504135241607FFEEDCCDB9A89A8B84C3
:1012220095A7B6C2D3E1F008192B3A4E5F6D7C94B4
:1012320085B7A6D2C3F1E018093B2A5E4F7D6CA5A3
:10124200B48697E3F2C0D129380A1B6F7E4C5DB594
:10125200A49687F3E2D0C139281A0B7F6E5C4DC683
:10126200D7E5F48091A3B24A5B69780C1D2F3ED674
:10127200C7F5E49081B3A25A4B79681C0D3F2EE763
:10128200F6C4D5A1B082936B7A48592D3C0E1FF754
:10129200E6D4C5B1A092837B6A58493D2C1E0F004B
:1012A20089129B24AD36BF48C15AD36CE57EF781C3
:1012B20008931AA52CB73EC940DB52ED64FF7602B3
:1012C2008B109926AF34BD4AC358D16EE77CF583A3
:1012D2000A9118A72EB53CCB42D950EF66FD740493
:1012E2008D169F20A932BB4CC55ED768E17AF38583
:1012F2000C971EA128B33ACD44DF56E960FB720673
:101302008F149D22AB30B94EC75CD56AE378F18762
:101312000E951CA32AB138CF46DD54EB62F9700852
:10132200811A932CA53EB740C952DB64ED76FF8942
:10133200009B12AD24BF36C148D35AE56CF77E0A32
:101342008318912EA73CB542CB50D966EF74FD8B22
:10135200029910AF26BD34C34AD158E76EF57C0C12
:10136200851E9728A13AB344CD56DF60E972FB8D02
:10137200049F16A920BB32C54CD75EE168F37A0EF2
:10138200871C952AA338B146CF54DD62EB70F98FE2
:0F139200069D14AB22B930C74ED55CE36AF178E3
:103D560052668D0000000000000000000000000018
:053D6600000000000058
:013DDC0022C4
:0300230002272988
:0B272900C0E0C083C082C0D075D01893
:102734002098030227F5755201AF99200225BF02A4
:102744001DD291301110AE0E050E74AE2EF582E43A
:102754003467F583EFF0750905D2020227F3C291BD
:102764000227F3300F14C20FAE0E050E74AE2EF511
:1027740082E43467F583EFF08072BF0917301110DB
:10278400AE0E050E74AE2EF582E43467F583EFF0D9
:10279400D20F8058BF0218530E8030114FAE0E0571
:1027A4000E74AE2EF582E43467F583EFF0803DEFCE
:1027B40064037028301110AE0E050E74AE2EF5822F
:1027C400E43467F583EFF09067ACE50EF0630E80B8
:1027D400530E80C202D2087509008010AE0E050E99
:1027E40074AE2EF582E43467F583EFF0750905C203
:1027F4009830997030036B301007309704D2008002
:10280400619066A1E0FFE510C39F4011C203D2149A
:10281400C290200B02D216C20BD2968045AF10058F
:102824001074AE2FF582E43468F583E0F5113009B5
:102834001953117F30012820D0082004226311800D
:10284400801D30041A6311808015300112E5115285
:1028540011300406A2D0929B8005A2D0B3929B852E
:062864001199C299D2AFE8
:09286A00D0D0D082D083D0E0323E
:1030EB007BFF7A0E79D21218493011147530FF75A7
:1030FB0031117532997BFF7A0F792D121849801295
:10310B007530FF75311175329D7BFF7A0F792D125A
:10311B0018499069AEE0FEA3E0FFC3E49FFFE49E75
:10312B00FEAB07FA3395E0F9F87F007E8C7D0A7CC5
:10313B0000121BAA8F338E328D318C307BFF7A0FAE
:10314B0079461218497BFF7A0F799EA210E433F56A
:10315B00301218497BFF7A0F79D4850A301218493F
:10316B007BFF7A107900A209E433F5301218497B02
:10317B00FF7A107921A201E433F5301218497BFF55
:10318B007A10794AA204E433F5301218497BFF7A9E
:10319B00107971A212E433F5301218497BFF7A10C3
:0C31AB00799CA20AE433F5301218492286
:102B7F007E107FCA1236C5EF4E70037F01227E1082
:102B8F007FCD1236C5EF4E6023123A1CA804A9055B
:102B9F00AA06AB077F007E8C7D0A7C00121BAA124F
:102BAF001C3C9069AEEEF0A3EFF0800A9069AE7412
:102BBF00FFF0A374B8F07E107FD31236C5EF4E60CE
:102BCF000C123D6CEF24D024FF92108002C2107EB5
:102BDF00107FD91236C5EF4E6007123A1C8F0A804C
:102BEF0003E4F50A7E107FDF1236C5EF4E600C123C
:102BFF003D6CEF24D024FF92098002C2097E107F22
:102C0F00E51236C5EF4E600C123D6CEF24D024FF59
:102C1F0092018002C2017E107FEB1236C5EF4E602B
:102C2F000C123D6CEF24D024FF92048002C2047E6C
:102C3F00107FF11236C5EF4E600E123D6CEF24D0AF
:102C4F0024FF920592128004C205C2127E107FF8F3
:102C5F001236C5EF4E600E123D6CEF24D024FF925A
:0C2C6F0005920A8004C205C20A7F002200
:1033ED00C203C216C208C202C20FE4F5109066A154
:1033FD00F0F50EF552C200D297D296750CFF90677C
:10340D00ADF075080CC206C21590669F7409F0A345
:10341D00F0750F05C209C204C201C213C210D20C4D
:10342D00E4F50AF509D2149069AE74FFF0A374B8EF
:10343D00F0C20AC205C212E4F50D122B7FE49067AB
:10344D00A2F0C2ADF5C9D2CDD2CCC2C9C2CAF5CD9A
:10345D00F5CC9069AEE0F5CBA3E0F5CA85CBCD8573
:10346D00CACCE4F59830010C2009095387BFD29FCF
:10347D00D29E8002D29E438740C29FC2ACC298C2E8
:0E348D009975B81075B710D2CAD29CD2AC2275
:103D8600E5136FFF9012A1936512F513EF9011A141
:033D960093F51290
:013D99002207
:013DDD0022C3
:0425D5008E298F2A92
:1025D900E4F52BF513F512AA06A9077B018B2F8ABF
:1025E9003089319067A2E0121B5C74012531F53105
:1025F900E43530F53030050F9067A3E0AB2FAA30F2
:10260900A931121B5C800D9066A0E0AB2FAA30A9FE
:1026190031121B5C752F01852930852A310D0DE496
:10262900FEEEC39D5018AB2F0531E531AA3070027B
:10263900053014F9121B43FF123D860E80E3AB2FC0
:102649000531E531AA307002053014F9E513121B82
:102659005CAB2FAA30A931E512121B5C0D0D752D4B
:1026690068752EAE752F01852930852A31852E8210
:10267900852D837402F0052EE52E7002052D052B9C
:10268900E4FEEEC39D504EAB2FAA30A931121B4375
:10269900F52C6402600BE52C64036005E52CB40994
:1026A90013852E82852D837409F0052EE52E70027F
:1026B900052D052B852E82852D83E52CF0052EE52C
:1026C9002E7002052D052B74012531F531E43530C5
:1026D900F5300E80AD852E82852D837403F0052E8D
:1026E900E52E7002052D052B906693E0FCA3E0FD15
:1026F900A3E0FEA3E0FFE4FAF9F8EF2401FFEA3EC4
:10270900FEE93DFDE83CFC906693121C5B30250D0B
:0F2719007E107FFF7C687DAEAB2B122873AF2B39
:01272800228E
:10328100E4FF9066A0E0FE7D000FED2405F582E4E9
:103291003461F583EEF00F74052401F582E43461A5
:1032A100F583E4F07C667D92FEED1DAA0470011C9D
:1032B100F5828A83E0FBAA070F74052AF582E434BC
:1032C10061F583EBF00EBE04E07C667D96E4FEEDD5
:1032D1001DAA0470011CF5828A83E0FBAA070F7402
:1032E100052AF582E43461F583EBF00EBE04E07C3F
:1032F100667D9AE4FEED1DAA0470011CF5828A83A5
:10330100E0FBAA070F74052AF582E43461F583EB2B
:10331100F00EBE04E07C667D9EE4FEED1DAA047005
:10332100011CF5828A83E0FBAA070F74052AF58246
:0B333100E43461F583EBF00EBE04E015
:01333C00226E
:0A3DC900C2992099FDD299D29022F0
:093DD300D2CAD29CD2ACC2082273
:103BD000AD072011337E677FA21225D59066A1EF35
:103BE000F0D203E4F51030250D7E117F0E7C687D48
:103BF000AEE0FB122873C296301003D20022E50A11
:093C00006003F54F22123DC922B8
:103AD5008F2820115430030F30254E7E117F1AE4B4
:103AE500FBFDFC12287322906378E09066A0F0300D
:103AF5000C117E637F77E52824FCFD1225D59066A1
:103B0500A1EFF0A21282055005750B05D215E4F55B
:103B150010D203C296301004D200800BE50A60046F
:0A3B2500F54F8003123DC9C21622BD
:10214100200603300B037F00222008030222D23035
:1021510011037F0022C208C291E4906475F0906778
:10216100ACE0FF547F24FCF528906476F090667A09
:10217100E0906477F0EF5480FF24AFF582E4346798
:10218100F583E0906478F074AE2FF582E43467ADA6
:1021910082FCE4F513F512FE9067ACE0547FF9EE92
:1021A100C39950140DEDAA0470010C14F5828A83B1
:1021B100E0FF123D860E80E0E512451360443025B4
:1021C100197E117F289067ACE0548024AEF582E43B
:1021D1003467AD82FCAB01122873906697E0FCA3D3
:1021E100E0FDA3E0FEA3E0FFE4FAF9F8EF2401FF2C
:1021F100EA3EFEE93DFDE83CFC906697121C5B025D
:1022010022D23005249067ACE05480FF24AEF582E1
:10221100E43467F583E09067A2F074AF2FF582E4B0
:102221003467F583E09067A3F0E5287039C215F5AE
:102231000B9067A3E0B4E01E7490F0200503022226
:10224100D2D2062025030222D27E117F37E4FBFD84
:10225100FC122873807B3025787E117F4DE4FBFDD5
:10226100FC122873806B9067ACE0548024B0F58237
:10227100E43467F58363A20190647963A201AF2816
:10228100121E8F30251C7E117F569067ACE0FB54E7
:102291008024AEF582E43467AD82FCEB547FFB12FF
:1022A100287390668FE0FCA3E0FDA3E0FEA3E0FFAE
:1022B100E4FAF9F8EF2401FFEA3EFEE93DFDE83CCE
:1022C100FC90668F121C5BA20A82055002D206D2D4
:0B22D10017301705C2177F01227F00A5
:0122DC0022DF
:103C410030082FC208C2913011289067ACE0FF54B0
:103C51008024AEF582E43467F58363A2019069B4F0
:103C610063A201EF547FFF121E8F9067ACE0547F77
:053C7100FF227F00228C
:05001E00C2AEC2AC22DD
:102A7E003018469080E8E0700F1239B93025077E85
:102A8E00117F65122D6BC2119080E8E0B40E12908A
:102A9E0080037408F03025077E117F6E122D6BC2F5
:102AAE00119080E8E0B4060F20110C3025077E113E
:102ABE007F79122D6BD211C21830116420030712C8
:102ACE002F348F288003E4F528E528603130250C5B
:102ADE007E117F8F7C697DB4FB1228739069B4637D
:102AEE00A2019068AE63A201AF28121E8F9066A15C
:102AFE00E528F0E4F510D290D203C296D299123C9A
:102B0E00419067ACEFF06018E0FF122C7B3025107F
:102B1E007E117F947C697DB49067ACE0FB122873C4
:102B2E00300008209705C200123DC9E54FB40106DA
:102B3E00E4F54F123DC9302625C226E509600DD5B4
:102B4E00090A630E80530E80C202C29130120FE545
:102B5E000B600BD50B08E4F510D203750B05A20A1A
:102B6E008206500C200309E4FF123BD0C206D20BA2
:012B7E002234
:103D9A003011037F0022301608201505C2167F0154
:043DAA00227F002252
:103B2F009080007480F090633663A201F583F58274
:103B3F0063A2017F08121E8F90633E63A2019080E3
:103B4F008863A2017F0A121E8F9080927407F0A3E0
:103B5F0074D0F0A37406F0906348E0FF9080B1F04A
:103B6F009080E1EFF09080957455F0A3F090800075
:0A3B7F007401F090800974F0F02248
:10394B00908009E04410F09080A0E070609080A11E
:10395B007482F09080A874FFF0A3F0A3F0A3F07F23
:10396B00039080AEEFF0A374CBF09080007402F064
:10397B00906AB4121C6700000000906AB4E090805B
:10398B0040F0906AB5E0908041F0906AB6E090808C
:10399B0042F0906AB7E0908043F0A3E4F0A3F0A369
:0D39AB00F0A3F0908018F0A3F0A3F0A3F0BB
:0139B80022EC
:103A7900908009E04440F09080D17482F07F0390F7
:103A890080DEEFF0A374CCF09080027402F0906AAB
:103A9900B8121C6700000000906AB8E0908058F0E6
:103AA900906AB9E0908059F0906ABAE090805AF033
:103AB900906ABBE090805BF0A3E4F0A3F0A3F0A3CD
:0B3AC900F0908030F0A3F0A3F0A3F019
:013AD40022CF
:1038D100908009E04420F09080B8E0706C9080B94D
:1038E1007482F07F039080C6EFF07FCDA3EFF07F6D
:1038F100039080C4EFF0A374CDF09080C074FFF00A
:10390100A3F0A3F0A3F09080017402F0906ABC12BE
:103911001C6700000000906ABCE090804CF0906A47
:10392100BDE090804DF0906ABEE090804EF0906ACC
:10393100BFE090804FF0A3E4F0A3F0A3F0A3F090D8
:093941008024F0A3F0A3F0A3F030
:01394A00225A
:1037CF008C288D29A907EAFDE975F018A424ACFF10
:1037DF00E5F034808F82F583EDF0EBFDE975F0189D
:1037EF00A4FFAEF024ACFBEE34808B82F583A3ED07
:1037FF00F08529828C83E0FDEF24A8FFEE3480FE54
:10380F008F82F583EDF08529828C83A3E08F828EE2
:10381F0083A3F0852982852883A3A3E0FDE975F0B2
:10382F0018A424A8FFE5F03480FE8F82F583A3A3AC
:10383F00EDF08529828C83A3A3A3E08F828E83A3CF
:04384F00A3A3F0221D
:0635B7008D2DAB07AA06F2
:1035BD00908000E030E5079065787401F022906A04
:1035CD00B4E0FCA3E0FDA3E0FEA3E0F5318E308D69
:1035DD002F8C2EAE02AF038E838F8263A201E53056
:1035ED00540744C0F58385318263A201AF2D121FAC
:1035FD0001E4FCFDFEE531252DF531EE3530F530DC
:10360D00ED352FF52FEC352EF52E908040E52EF073
:10361D00A3E52FF0A3E530F0A3E531F09080007421
:10362D0020F0AF31AE30AD2FAC2E906AB4121C5BD2
:01363D00226A
:06363E008D28AB07AA066F
:10364400908002E030E5079065787403F022906A78
:10365400B8E0FCA3E0FDA3E0FEA3E0F52C8E2B8DE7
:103664002A8C29AE02AF038E838F8263A201E52BDD
:10367400540744D0F583852C8263A201AF28121F1E
:1036840001E4FCFDFEE52C2528F52CEE352BF52B6D
:10369400ED352AF52AEC3529F529908058E529F0ED
:1036A400A3E52AF0A3E52BF0A3E52CF090800274A7
:1036B40020F0AF2CAE2BAD2AAC29906AB8121C5B5B
:0136C40022E3
:02333D008F28D7
:10333F00908001E030E5099065787402F07F0022FB
:10334F00906ABCE0FCA3E0FDA3E0FEA3E0F52C8EA9
:10335F002B8D2A8C2990667B63A201E52B540744A1
:10336F00C8F583852C8263A2017F06121F17E52CF7
:10337F002406F52CE4352BF52BE4352AF52AE43514
:10338F0029F52990657963A201E52B540744C8F507
:10339F0083852C8263A201AF28121F17E4FCFDFE68
:1033AF00E52C2528F52CEE352BF52BED352AF52AB6
:1033BF00EC3529F52990804CE529F0A3E52AF0A3F7
:1033CF00E52BF0A3E52CF09080017420F0AF2CAE2C
:0D33DF002BAD2AAC29906ABC121C5BAF28F4
:0133EC0022BE
:10297A009081E0E0F528052805280528052805287E
:10298A0005280528052805280528908010E0F52B3C
:10299A00A3E0F52CA3E0F52DA3E0F52E9081E1E06C
:1029AA00F5280528052805280528052805280528C5
:1029BA00052805280528908014E0F52FA3E0F530B6
:1029CA00A3E0F531A3E0F532E531B52D08E532B5DE
:1029DA002E037F0022E4F528E531540744E0F5830D
:1029EA0085328263A20190637563A2017F08121F78
:1029FA004790637763A2019062AE63A2017F0612D9
:102A0A001E8F906375E0F529A3E0F52AE4F5289076
:102A1A006375E0702AA3E024F8F528E531540744E9
:102A2A00E0F58385328274082582F582E43583F5E0
:102A3A008363A20190637563A201AF28121F47AE98
:102A4A0029E4FCFDE532252AF532E5313EF531ED82
:102A5A003530F530EC352FF52F908014E52FF0A3A3
:102A6A00E530F0A3E531F0A3E532F0908000744040
:032A7A00F0AF2892
:012A7D002236
:1022DD009081E6E0F528052805280528052805281C
:1022ED0005280528052805280528908028E0F52BC8
:1022FD00A3E0F52CA3E0F52DA3E0F52E9081E7E00A
:10230D00F528052805280528052805280528052868
:10231D0005280528052890802CE0F52FA3E0F53041
:10232D00A3E0F531A3E0F532E4F528E531B52D0A4A
:10233D00E532B52E05C220022449E531540744F09B
:10234D00F58385328263A20190637563A2017F08D4
:10235D00121F47906375E0F529A3E0F52AE52A459C
:10236D002970099080027410F07F0022906682E03F
:10237D00FFF46030906377E06F6003022410906685
:10238D0083E0FF906378E06F7079906684E0FF9052
:10239D006379E06F706D906685E0FF90637AE06F12
:1023AD006031805F906377E0906682F0906378E0B3
:1023BD00906683F0906379E0906684F090637AE0A4
:1023CD00906685F090637BE0FFA3E0906349CFF0CA
:1023DD00A3EFF0906375E0702AA3E024F8F528E5EB
:1023ED0031540744F0F58385328274082582F582D5
:1023FD00E43583F58363A20190637563A201AF2871
:10240D00121F47AE29E4FCFDE532252AF532E531F0
:10241D003EF531ED3530F530EC352FF52FAF2EAED5
:10242D002DAD2CAC2BAB32AA31A930A82FD3121C59
:10243D004A40099080027410F07F002290802CE5B4
:10244D002FF0A3E530F0A3E531F0A3E532F0908055
:06245D00027440F0AF28FC
:012463002256
:102464009081E3E0F5280528052805280528052896
:102474000528052805280528052890801CE0F52B4B
:10248400A3E0F52CA3E0F52DA3E0F52E9081E4E084
:10249400F5280528052805280528052805280528E0
:1024A400052805280528908020E0F52FA3E0F530C5
:1024B400A3E0F531A3E0F532E4F528E531B52D0AC2
:1024C400E532B52E05C2210225BAE531540744E8A8
:1024D400F58385328263A20190600463A2017F0EBA
:1024E400121F5D906004E0F529A3E0F52A90600CCA
:1024F400E0FFF4604A90667BE0FEEF6E7079A3E043
:10250400FF90600DE06F706F90667DE0FF90600E4D
:10251400E06F706390667EE0FF90600FE06F70572D
:1025240090667FE0FF906010E06F704B906680E0F3
:10253400FF906011E06F703FE4906013F0800890AA
:10254400601374FFF0D2D9906004E0702AA3E024F1
:10255400F2F528E531540744E8F583853282740E98
:102564002582F582E43583F58363A20190600463D8
:10257400A201AF28121F5DAE29E4FCFDE532252A35
:10258400F532E5313EF531ED3530F530EC352FF5EA
:102594002FAF2EAE2DAD2CAC2BAB32AA31A930A867
:1025A4002FD3121C4A5006E52A4529700990800150
:1025B4007410F07F0022908020E52FF0A3E530F026
:1025C400A3E531F0A3E532F09080017440F0AF2828
:0125D40022E4
:042D6B008E2D8F2EEC
:102D6F00908000E030E5079065787401F022906A5A
:102D7F00B4E0FCA3E0FDA3E0FEA3E0F5348E338DB9
:102D8F00328C31E534FFE5335407FEE42FF530EE96
:102D9F0034C0F52F853082F5837423F00530E5308C
:102DAF007002052F532FC7F582852F83740AF00504
:102DBF0030E5307002052F532FC790633E63A20199
:102DCF00852F8385308263A2017F06121F0174064F
:102DDF002530F530E4352FF52F852D83852E826331
:102DEF00A201852F8385308263A201121EE5E4FCC8
:102DFF00FDFE906AB4E0F8A3E0F9A3E0FAA3E02F98
:102E0F00FFEE3AFEED39FDEC38FCEF2408FFE43E0F
:102E1F00FEE43DFDE43CFC906AB4121C5B906AB486
:102E2F00E0908040F0906AB5E0908041F0906AB6F3
:102E3F00E0908042F0906AB7E0908043F09080007D
:032E4F007420F0FC
:012E5200225D
:0A2873008E328F338C348D358B3696
:10287D00908000E030E5079065787401F022906A51
:10288D00B4E0FCA3E0FDA3E0FEA3E0F53C8E3B8DA0
:10289D003A8C39E53CFFE53B5407FEE42FF538EE65
:1028AD0034C0F537853882F5837423F00538E53863
:1028BD00700205375337C7F582853783740AF005E3
:1028CD0038E538700205375337C790633E63A20170
:1028DD0085378385388263A2017F06121F01740636
:1028ED002538F538E43537F53785328385338263FE
:1028FD00A20185378385388263A201121EE58F3DC3
:10290D00EF2538F538E43537F537E536601785347A
:10291D008385358263A20185378385388263A20161
:10292D00AF36121F01E53D24082536F536FFE4FCD0
:10293D00FDFEE53C2FF53CEE353BF53BED353AF52F
:10294D003AEC3539F539908040E539F0A3E53AF0A8
:10295D00A3E53BF0A3E53CF09080007420F0AF3C84
:0C296D00AE3BAD3AAC39906AB4121C5B72
:01297900223B
:063010008E468F478D483B
:10301600908000E030E5079065787401F022906AB0
:10302600B4E0FCA3E0FDA3E0FEA3E0F54E8E4D8DDB
:103036004C8C4BE54EFFE54D5407FEE42FF54AEE6A
:1030460034C0F549854A82F5837423F0054AE54A7A
:10305600700205495349C7F582854983EBF0054A55
:10306600E54A700205495349C790633E63A201854C
:103076004983854A8263A2017F06121F01740625D1
:103086004AF54AE43549F54985468385478263A270
:1030960001854983854A8263A201AF48121F0174E4
:1030A600082548F548FFE4FCFDFEE54E2FF54EEEFB
:1030B600354DF54DED354CF54CEC354BF54B9080DB
:1030C60040E54BF0A3E54CF0A3E54DF0A3E54EF04B
:1030D6009080007420F0AF4EAE4DAD4CAC4B906A74
:0430E600B4121C5BA9
:0130EA0022C3
:02374A008F41AD
:10374C00908000E030E5079065787401F022906A73
:10375C00B4E0FCA3E0FDA3E0FEA3E0F5458E448DB0
:10376C00438C42E545FFE5445407FEE42FFFEE345D
:10377C00C09062B463A201F5838F8263A201AF4152
:10378C00121F01E4FCFDFEE5452541F545EE3544EF
:10379C00F544ED3543F543EC3542F542908040E578
:1037AC0042F0A3E543F0A3E544F0A3E545F0908097
:1037BC00007420F0AF45AE44AD43AC42906AB412F5
:0237CC001C5B84
:0137CE0022D8
:062E53008E288F29AB055B
:102E5900908000E030E5079065787401F022906A6F
:102E6900B4E0FCA3E0FDA3E0FEA3E0F52F8E2E8DD8
:102E79002D8C2CE52FFFE52E5407FEE42FF52BEEC4
:102E890034C0F52A852B82F5837423F0052BE52BB5
:102E99007002052A532AC7F582852A83EBF0052B90
:102EA900E52B7002052A90633E63A201852A83857A
:102EB9002B8263A2017F06121F017406252BF52BB5
:102EC900E4352AF52A532AC7E528852B82852A83E2
:102ED900F0052BE52B7002052A532AC7F582852AAE
:102EE90083E529F0052BE52B7002052A532AC7E54E
:102EF9002F240AF52FE4352EF52EE4352DF52DE492
:102F0900352CF52C908040E52CF0A3E52DF0A3E5B8
:102F19002EF0A3E52FF09080007420F0AF2FAE2E95
:0A2F2900AD2DAC2C906AB4121C5BB5
:012F3300227B
:1039B900908009E04480F09080E97441F07F09909B
:1039C90080F6EFF0A37464F09080037402F09080A5
:1039D90003E020E1F99069B0121C67000000009033
:1039E90069B0E0908064F09069B1E0908065F090F2
:1039F90069B2E0908066F09069B3E0908067F0A3C7
:103A0900E4F0A3F0A3F0A3F090803CF0A3F0A3F0BE
:023A1900A3F018
:013A1B002288
:102F34009081E9E0F52905290529052905290529AF
:102F440005290529052905290529908034E0F52A54
:102F5400A3E0F52BA3E0F52CA3E0F52D9081EAE0A6
:102F6400F5290529052905290529052905290529FD
:102F7400052905290529908038E0F52EA3E0F52FD1
:102F8400A3E0F530A3E0F531E530B52C08E531B523
:102F94002D037F0022AF31AE30AD2FAC2EAB2DAA66
:102FA4002CA92BA82AD3121C4A400AAF31AE2DEE0D
:102FB4009FF529800AAF31EFF404AE2D2EF529E5F3
:102FC40030540744E0F58385318263A2019069B4EB
:102FD40063A201AF29121F75E4FCFDFEE53125292A
:102FE400F531EE3530F530ED352FF52FEC352EF586
:102FF4002E908038E52EF0A3E52FF0A3E530F0A362
:0B300400E531F09080037440F0AF292C
:01300F00229E
:022C7B008F299F
:102C7D009080E8E0640660037FFF229069B0E0FC7D
:102C8D00A3E0FDA3E0FEA3E0F52D8E2C8D2B8C2A69
:102C9D00E4FFFEFDFCAB2DAA2CA92BA82AC3121C08
:102CAD004A70609081F9E0F52A9069B0E0FCA3E0EC
:102CBD00FDA3E0FEA3E0FFE4FAF9F8EF2401FFEA3B
:102CCD003EFEE93DFDE83CFC9069B0121C5B90694D
:102CDD00B0E0FCA3E0FDA3E0FEA3E0FFE4F8EF24E9
:102CED0001FFEA3EFEE93DFDE83CFC9069B0121C97
:102CFD005B908064E0F52AA3E0F52BA3E0F52CA30F
:102D0D00E0F52D9069B463A201E52C540744D8F584
:102D1D0083852D8263A201AF29121F2FE4FCFDFED6
:102D2D00E52D2529F52DEE352CF52CED352BF52B37
:102D3D00EC352AF52A908064E52AF0A3E52BF0A363
:102D4D00E52CF0A3E52DF09080037420F0AF2DAEAF
:0D2D5D002CAD2BAC2A9069B0121C5B7F00DE
:012D6A002246
:0A3DBE00E4FEEEC39F50030E80F8F0
:013DC80022D8
:103D1600A2AF9228C2AF438E2075D2028F828E83C5
:0C3D2600E0FFE4F5D2538EDFA22892AF3C
:013D3200226E
:103CAA00E5D220E0FBA2AF9228C2AF43D2028F82B4
:103CBA008E83EDF075D25063D250A22892AFE5D22E
:033CCA0020E0FBFC
:013CCD0022D4
:10385300E4FDED2401FFE433FE123D1674362DF52D
:1038630082E43463F583EFF00DBD3FE6E4FDED2420
:103873007FFFE433FE123D16742D2DF582E434618F
:10388300F583EFF0742D2DF582E43461F583E07058
:103893001B742D2DF582E43461F5837420F0742EAE
:1038A3002DF582E43461F583E4F080040DBD80BE20
:1038B300E49061ACF0FDEDFF7E00123D1674AD2D7A
:0D38C300F582E43461F583EFF00DBDFEE900
:0138D00022D5
:023C76008B2D94
:103C7800A2AF9228C2AF85A22E53A2FE8E838F8256
:103C880005A28C838D827409121F8BE52D53A2FE29
:103C980043A220121F8D53A2DF852EA2A22892AF25
:013CA800FF1C
:013CA90022F8
:103D3300A2AF9228C2AF8C838D82EF121F8B43A256
:0C3D430020121F8D53A2DFA22892AFFFB8
:013D4F002251
:023CCE008F283D
:103CD000A2AF9228C2AFE4F5838D827406121F8BC7
:103CE000E52843A220121F8D53A2DFA22892AF7FA6
:013CF00001D2
:013CF10022B0
:023CF2008F2819
:103CF400A2AF9228C2AFE4F5838D82740A121F8B9F
:103D0400E52843A220121F8D53A2DFA22892AF7F81
:013D140001AD
:013D1500228B
:101DB400A907E7FFA805EF93C3966008403B74FCAE
:101DC4002FFF80F00F08EF93C3966008402B74FB3D
:101DD4002FFF80E00F08EF93C3966008401B74FA4E
:101DE4002FFF80D00F08EF93D3966008400B74F94F
:101DF4002FFF80C01F1F1F1F1FEF54FEF80303F7A0
:101E0400E893FC08E893FD08E893FE08E893FF22B2
:101E140009E993C39D6008402974FB29F980F109FD
:101E2400E993C39E6008401A74FA29F980E209E92B
:101E340093D39F6008400B74F929F980D3191919B9
:101E44001919E9C313C313FF22740093F8ECC39860
:101E54004024701F740193F8EDC3984019701474F2
:0E1E64000293F8EEC398400E7009740393F8D1
:101E7200EFC39840037F00227F0122EDF8E6F008CD
:101E8200A3DFFA22EDF8E0F608A3DFFA22E0A3636B
:101E9200A201F0A363A201DFF475A2002263A201F2
:101EA200F0A363A20122E0A363A201F0A363A20153
:101EB200E0A363A201F0A363A201E463A201F0A381
:101EC20063A201DFE175A20022E0A363A2016DFE1D
:101ED200936CFDEE058393FC158363A201DFEA7523
:101EE200A200227F00E493A363A201F00F600CA37F
:101EF200E583C2E3F58363A20180EA75A20022E0D2
:101F0200A363A201F0A3E583C2E3F58363A201DF29
:101F1200EE75A20022E0A363A201F0A3E583C2E46E
:101F2200D2E3F58363A201DFEC75A20022E0A36392
:101F3200A201F0A3E58344F8C2E5F58363A201DFC1
:101F4200EC75A20022E583C2E3F583E0A363A2015C
:101F5200F0A363A201DFEE75A20022E583C2E4D200
:0A1F6200E3F583E0A363A201F0A3FE
:101F6C0063A201DFEC75A20022E58344F8F583E05F
:101F7C00A363A201F0A363A201DFEE75A20022F914
:101F8C0022C002C004C00612FFF0D006D004D0025A
:011F9C002222
:10353700020869E493A3F8E493A34003F68001F239
:1035470008DFF48029E493A3F85407240CC8C33395
:10355700C4540F4420C8834004F456800146F6DF64
:10356700E4800B0102040810204080903D50E47E67
:10357700019360BCA3FF543F30E509541FFEE49359
:10358700A360010ECF54C025E060A840B8E493A320
:10359700FAE493A3F8E493A3C8C582C8CAC583CA4B
:1035A700F0A3C8C582C8CAC583CADFE9DEE780BE03
:013D6B000057
:101B4300BB010689828A83E0225002E722BBFE02A0
:091B5300E32289828A83E49322D3
:101B5C00BB010689828A83F0225002F722BBFE0168
:021B6C00F32262
:101B6E0075F008758200EF2FFFEE33FECD33CDCC2E
:101B7E0033CCC58233C5829BED9AEC99E5829840B1
:101B8E000CF582EE9BFEED9AFDEC99FC0FD5F0D68E
:101B9E00E4CEFBE4CDFAE4CCF9A88222B800C1B9B8
:101BAE000059BA002DEC8BF084CFCECDFCE5F0CBF6
:101BBE00F97818EF2FFFEE33FEED33FDEC33FCEB2F
:101BCE0033FB10D703994004EB99FB0FD8E5E4F9EA
:101BDE00FA227818EF2FFFEE33FEED33FDEC33FCD7
:101BEE00C933C910D7059BE99A4007EC9BFCE99ACB
:101BFE00F90FD8E0E4C9FAE4CCFB2275F010EF2F10
:101C0E00FFEE33FEED33FDCC33CCC833C810D7070F
:101C1E009BEC9AE899400AED9BFDEC9AFCE899F84A
:0E1C2E000FD5F0DAE4CDFBE4CCFAE4C8F922DD
:0E1C3C00C3E49FFFE49EFEE49DFDE49CFC22B9
:101C4A00EB9FF5F0EA9E42F0E99D42F0E89C45F0F0
:011C5A002267
:0C1C5B00ECF0A3EDF0A3EEF0A3EFF022FC
:101C6700A8828583F0D083D082121C7E121C7E123C
:101C77001C7E121C7EE473E493A3C583C5F0C58361
:101C8700C8C582C8F0A3C583C5F0C583C8C582C8C7
:011C9700222A
:1017E700E53C2430F8E6053C22782D302F0278308E
:1017F700E475F001121D14021B432028EB7F2ED243
:10180700288018EF540F2490D43440D4FF302C0B89
:10181700EF24BFB41A0050032461FFE53D600215B1
:101827003D0540E5407002053F302F0D782DE475EA
:10183700F001121D14EF021B5C023B897403D22FC7
:101847008003E4C22FF53C8B2D8A2E892FE4F53DCA
:10185700F53FF540E53D60077F2012182280F575BA
:101867003EFFC229C228C22AC22BC22DC22EC230B5
:101877001217F0FF700D302F057F00121833AF409D
:10188700AE3F22B4255FC2D5C22C1217F0FF24D079
:10189700B40A00501A75F00A783D30D50508B6FF2E
:1018A7000106C6A426F620D5047002D22B80D924BF
:1018B700CFB41A00EF5004C2E5D22C021A33D22952
:1018C70080C6D22880C0D22A80BCD2D580BAD22D79
:1018D70080B47F20121822202A077401B53D0040EA
:1018E700F11217E7FF12182202185BD230D22E80AE
:1018F700951217E7FB1217E7FA1217E7F94A4B7029
:101907000679047A1B7BFF202A2EE53D602A7E009C
:101917008E82758300121C9860060EEE653E70F08D
:10192700C2D5EBC0E0EAC0E0E9C0E0EE121A7AD017
:10193700E0F9D0E0FAD0E0FB121B43FF60AAEBC04E
:10194700E0EAC0E0E9C0E0121822D0E02401F9D0B3
:10195700E03400FAD0E0FBE53E0460DCD53ED980F8
:10196700877BFF7A1A7976D22A809C791080027950
:1019770008C22EC2308008D2D5790A8004790AC2FB
:10198700D5E53E047002F53EE4FAFDFEFF1217E7C7
:10199700FC7B082029131217E7FD7B1030280A1259
:1019A70017E7FE1217E7FF7B20EC3382D592D5505D
:1019B70013C3E43028069FFFE49EFEE42029039D1D
:1019C700FDE49CFCE4CBF8C229EC700CCFCECDCC67
:1019D700E824F8F870F38017C3EF33FFEE33FEED1A
:1019E70033FDEC33FCEB33FB994002FB0FD8E9EBFB
:1019F700302905F8D0E0C448B229C0E00AEC4D4EC2
:101A07004F78207B0070C2EAB53E0040BCC0E012B0
:101A17001A7CD0F0D0E0202904C4C0E0C4B229C0A9
:101A2700F012180BD0F0D5F0EB02185B121D7318EB
:101A3700F85319725818C94C18C54219764F197EB0
:0F1A470044197E4918DE431984551968461968F9
:101A5600451968471B245018CD2D18D12E18F42B84
:101A660018D52318F2201B0D2A188D48000018ECF3
:101A76003F3F3F00790AA2D5202B14302D09B9101B
:101A8600020404B9080104A2D5202E025001042044
:101A96002A68922AB53D005034C0E07F20302B19C9
:101AA6007F30A22A722E722D500F121AD3C22AC26A
:101AB6002EC22DC2307F30800F302D03E9C0E012D8
:101AC6001822302D03D0E0F9D0E0B53DCC302D17EB
:101AD6007F30B9100C1218227F58302C077F78807F
:101AE60003B90803121822302A057F2D0218227F17
:101AF600202030F87F2B202EF322922A80CF286ECA
:101B0600756C6C2900D2291217E73029F8C229789A
:101B16003D30D50108F602188D2D5043495812174D
:101B2600E72403B405004001E4901B1F9312181329
:0D1B3600743A121813D22B753D0402197277
:101F9D008B288A29892AE4F534F533F532F531F5A4
:101FAD002FF530E52C452D452B6012EBC0E0EAC036
:101FBD00E0E9C0E0AB2BAA2CA92D121D24AB2805FE
:101FCD002AE52AAA297002052914F9121B43F535B1
:101FDD00C394094007E535D3940D40E1E535642000
:101FED0060DBE535B42D054330038016E535B42BA4
:101FFD0005433001800C74FF252AF52A74FF35291D
:10200D00F529E52E60046410703FAB28AA29A92A92
:10201D00121B4364306009E52E702E752E0A80293F
:10202D00900001121C98FF64786004EFB4581343BC
:10203D003001752E107402252AF52AE43529F5296B
:10204D008007E52E7003752E08AB28052AE52AAA10
:10205D00297002052914F9121B43F535C39461400B
:10206D000AE535D3947A50035335DF74D02535F511
:10207D0035C3940A400CE5359411406D74F925353E
:10208D00F535E535D3952E506043300185343985CE
:10209D003338853237853136AF2E7E00E4FCFDAB0B
:1020AD0034AA33A932A831121CC5C8ECC8C9EDC970
:1020BD00CAEECACBEFCBE4FCFDFEEB2535F534EED5
:1020CD003AF533ED39F532EC38F531AF34AE33AD99
:1020DD0032FCAB39AA38A937A836D3121C4A5003A3
:1020ED00022056433004022056E53020E003E48000
:1020FD002DE52C452D452B601EAB28E52A24FFF937
:10210D00E52934FFFAEBC0E0EAC0E0E9C0E0AB2B13
:10211D00AA2CA92D121D24E53030E20774FFFFFE15
:10212D00FDFC22E530AF34AE33AD32AC3130E103DE
:04213D00021C3C2222
:101C9800BB010CE58229F582E5833AF583E0225001
:101CA80006E92582F8E622BBFE06E92582F8E2224B
:0D1CB800E58229F582E5833AF583E4932265
:101CC500E88FF0A4CC8BF0A42CFCE98EF0A42CFCBE
:101CD5008AF0EDA42CFCEA8EF0A4CDA8F08BF0A43C
:101CE5002DCC3825F0FDE98FF0A42CCD35F0FCEB9B
:101CF5008EF0A4FEA9F0EB8FF0A4CFC5F02ECD3960
:0F1D0500FEE43CFCEAA42DCE35F0FDE43CFC22CC
:101D1400FAE6FB0808E6F925F0F618E6CA3AF622D0
:101D2400BB011A89828A83D0F0D0E0F8D0E0F9D0E0
:101D3400E0FAD0E0FBE8C0E0C0F0021DA25016E9D2
:101D4400F8D083D082D0E0F9D0E0FAD0E0FBC082B2
:101D5400C083021D99BBFE16E9F8D083D082D0E07F
:0F1D6400F9D0E0FAD0E0FBC082C083021DAB22B1
:101D7300D083D082F8E4937012740193700DA3A3FF
:101D830093F8740193F5828883E473740293686013
:061D9300EFA3A3A380DF13
:091D9900EBF608EAF608E9F6226F
:091DA200EBF0A3EAF0A3E9F02242
:091DAB00EBF208EAF208E9F22269
:00000001FF
